:100000000C9460030C94A3030C94A3030C94A3031B
:100010000C94A3030C94A3030C94A3030C94A303C8
:100020000C94A3030C94A3030C94112C0C94B42AE9
:100030000C94A3030C94A3030C94A3030C94A303A8
:100040000C94A3030C94A3030C94A3030C94A30398
:100050000C94030D0C94A3030C94A3030C94B90308
:100060000C94A3030C94A3030C94A3030C94A30378
:100070000C94A3030C94A3030C94A3030C94A30368
:100080000C94A3030C94A3030C94A3030C94A30358
:100090000C94A3030C94A3030C94A3030C94A30348
:1000A0000C94A3030C94A3030C94A3032900140041
:1000B0001A000800150017001C0018000C001200A0
:1000C00013002A00E20004001600070009000A00DD
:1000D0000B000D000E000F0033002800E1001D0092
:1000E0001B00060019000500110010003600370043
:1000F0003800E30000000000000000002C442B4406
:100100002C00E000000000000000000035001E0090
:100110001F002000210022002300240025002600CB
:1001200027000000E200B748B648CD48B548E94886
:100130000000000000002F0030003400E1001D012D
:100140001B01E0011901EA48E248000000002D000F
:100150002E00E30000000000000000002D44FFFF1F
:100160004C00E000000000000000000005443A00E0
:100170003B003C003D000000650046004700480091
:1001800000000000E2003E003F004000410000008F
:10019000000049004A004B0000000000E10042005E
:1001A000430044004500000000004C004D004E009C
:1001B0003100E3000000000000000000FFFF2D44BC
:1001C0002B00E000000000000000000004440000DC
:1001D000000000000000470054005F006000610064
:1001E0002D000000E2004A0052004D004B00390093
:1001F00055005C005D005E0057002800E1005000E3
:1002000051004F004E000000620059005A005B0090
:100210000000E3000000000000000000FFFFFFFFFF
:100220000000E00000000000000000002ED12FD1EF
:1002300030D131D132D133D150D151D152D153D12A
:1002400054D155D1C0D134D136D138D13AD13ED1A3
:1002500043D147D149D14BD14DD14FD1C1D135D166
:1002600037D139D13BD13FD144D148D14AD14CD1FA
:100270004ED156D100000000000000003CD13DD11D
:1002800045D146D100000000000000001E001E0005
:100290001E001E001E001E001E001E001E001E006E
:1002A0001E001E00C0D114001A000800150017001F
:1002B0001C0018000C00120013002F00C1D1040014
:1002C0001600070009000A000B000D000E000F00C9
:1002D0003300340000000000000000000600190098
:1002E000110010000000000000000000302E31312D
:1002F0002E302B32370076657273696F6E0076652B
:100300007273696F6E0005010906A101050719E006
:1003100029E71500250175019508810295017508E9
:1003200081019505750105081901290591029501BD
:100330007503910195067508150025FF050719003D
:1003400029FF8100C0050C0901A1018504150026C3
:10035000FF0319002AFF03950475108100C00501F1
:100360000906A1018508050719E029E715002501FF
:10037000750195088102050819012908950875017C
:1003800091020507750495018101190429DD150005
:100390002501750195D98102750395018101C0057B
:1003A000010980A1018505150026FF00190029FF1C
:1003B000950175088100C06573636170655F6F6E3C
:1003C0006573686F742E63616E63656C5F6B6579CE
:1003D000006573636170655F6F6E6573686F742E1F
:1003E00063616E63656C5F6B657900457363617013
:1003F000654F6E6553686F740074726967676572E4
:10040000006D6170006D6163726F732E006D6163CA
:10041000726F732E6D61700A6D6163726F732E74EB
:100420007269676765720044796E616D69634D61D9
:1004300063726F7300656570726F6D2E65726173A4
:100440006500656570726F6D2E6672656500656525
:1004500070726F6D2E636F6E74656E747300656578
:1004600070726F6D2E636F6E74656E74730A65655E
:1004700070726F6D2E667265650A656570726F6D5C
:100480002E6572617365002F00637263007665727A
:1004900073696F6E0076616C69643F0064656661C4
:1004A000756C744C617965720073657474696E67FC
:1004B000732E0073657474696E67732E646566616C
:1004C000756C744C617965720A73657474696E67D2
:1004D000732E76616C69643F0A73657474696E6724
:1004E000732E76657273696F6E0A73657474696EC4
:1004F00067732E63726300637573746F6D00646558
:100500006661756C74006F6E6C79437573746F6D92
:10051000006B65796D61702E006B65796D61702E71
:10052000637573746F6D0A6B65796D61702E6465A8
:100530006661756C740A6B65796D61702E6F6E6C97
:1005400079437573746F6D00454550524F4D4B653F
:10055000796D61700066616C736500747275650019
:10056000706C7567696E73006465766963652E7279
:10057000657365740068656C700A646576696365A7
:100580002E72657365740A706C7567696E730068A6
:10059000656C70000D0A2E004D6F7573654B6579A3
:1005A00073004F6E6553686F740051756B65797396
:1005B00000537061636543616465740047656D69EC
:1005C0006E69505200080B0002020200000904008C
:1005D00000010202000005240010010524010101B0
:1005E00004240206052406000107058103100040CB
:1005F00009040100020A0000000705020240000091
:100600000705830240000012010002EF020140EDE5
:10061000FE6060000101020301534F46542F48520F
:1006200055460053706C69746F6772617068790029
:100630000403090405010902A10185010509190145
:100640002908150025019508750181020501093069
:10065000093109381581257F750895038106050C38
:100660000A38021581257F750895018106C00501AC
:100670000902A1010509190129081500250195089C
:100680007501810205010930093116000026FF7F3E
:1006900075109502810209381581257F750895012D
:1006A0008106C0002606D40CA20E3B0F2F108E1020
:1006B0001F164419A122AB241F26B92CAA2E7E2F67
:1006C00011241FBECFEFDAE0DEBFCDBF04B603FEBC
:1006D00018C08091F8049091F904A091FA04B091A7
:1006E000FB048730904BA740B04B59F41092F804AC
:1006F0001092F9041092FA041092FB04E0E0F8E37F
:10070000099511E0A0E0B1E0E2EEF0E602C005904C
:100710000D92AC3AB107D9F724E0ACEAB1E001C0E0
:100720001D92A83FB207E1F713E0C0E6D3E004C092
:100730002197FE010E94D92FC235D107C9F70E9427
:10074000A6030C946F300C94000008950E94780466
:100750000E94A50388E494E00E94892C0E94090667
:10076000C0E0D0E00E9420062097E1F30E94000044
:10077000F9CF1F920F920FB60F9211242F933F9330
:100780008F939F93AF93BF938091AD019091AE01F2
:10079000A091AF01B091B0013091AC0123E0230FE3
:1007A0002D3758F50196A11DB11D2093AC01809302
:1007B000AD019093AE01A093AF01B093B0018091D1
:1007C000B1019091B201A091B301B091B401019631
:1007D000A11DB11D8093B1019093B201A093B3010B
:1007E000B093B401BF91AF919F918F913F912F91A1
:1007F0000F900FBE0F901F90189526E8230F0296BA
:10080000A11DB11DD2CF2FB7F8946091AD017091A9
:10081000AE018091AF019091B0012FBF08953FB715
:10082000F8948091B1019091B201A091B301B0917F
:10083000B40126B5A89B05C02F3F19F00196A11D54
:10084000B11D3FBFBA2FA92F982F8827BC01CD011A
:10085000620F711D811D911D42E0660F771F881F79
:10086000991F4A95D1F708958F929F92AF92BF92A8
:10087000CF92DF92EF92FF926B017C010E940F04F6
:100880004B015C01C114D104E104F104E9F00E94C0
:10089000B82C0E940F04681979098A099B09683EDF
:1008A00073408105910570F321E0C21AD108E10877
:1008B000F10888EE880E83E0981EA11CB11CC114BB
:1008C000D104E104F10429F7FF90EF90DF90CF907D
:1008D000BF90AF909F908F9008958230910538F02F
:1008E000880F991F880F991F05970197F1F70895B1
:1008F000789484B5826084BD84B5816084BD85B5FB
:10090000826085BD85B5816085BDEEE6F0E08081C1
:1009100081608083E1E8F0E01082808182608083E2
:10092000808181608083E0E8F0E080818160808365
:10093000E1E9F0E080818260808380818160808352
:10094000E0E9F0E0808181608083E1ECF0E080818B
:1009500084608083808182608083808181608083E5
:10096000E3ECF0E0808181608083E0ECF0E0808166
:1009700082608083E2ECF0E0808181608083EAE73E
:10098000F0E08081846080838081826080838081C8
:1009900081608083808180688083089508958CE0E1
:1009A000ECE4F1E0DB0101900D928A95E1F78CE037
:1009B000089583EE93E00E94AF2481E493E00E94C7
:1009C000B9178CE793E00E94621F82EB93E00E94CC
:1009D000162382E191E00E94EF1D87E693E00E94DA
:1009E000B4198EED92E00E94F61080EE92E00E9423
:1009F000331380E0089587E393E00E941A1581E4A1
:100A000093E00E94AF1787E693E00E94C9198EED2C
:100A100092E00E94B61080E0089587E393E00E9480
:100A2000171680E00895CF93DF93EC01BC018CE7AB
:100A300093E00E94F221811107C0BE0182EB93E096
:100A4000DF91CF910C943324DF91CF910895CF9310
:100A5000DF93EC01BC0185E091E00E945F11811100
:100A60002CC0BE0183EE93E00E94C424811125C0F6
:100A70002B81822F90E0982F88272A81280F392FE9
:100A8000311DC901805C914D0297F8F44981309184
:100A9000B501205C81E090E001C0880F2A95EAF75B
:100AA00041FF0EC040FD0CC0832B8093B501833005
:100AB00019F480E00E94E40B81E0DF91CF9108956A
:100AC000809583238093B501F7CFBE0182E191E049
:100AD0000E94A51E8111F1CFBE0187E693E00E941E
:100AE0003F1A8111EACFBE0180EE92E0DF91CF91F3
:100AF0000C941013BC0187E693E00C94F9190F9342
:100B00001F93CF938C01BC0186E493E00E941719D8
:100B1000C82F81114BC0B80181E493E00E945B189B
:100B2000C82F811143C0B80185E393E00E943516B8
:100B3000C82F81113BC0B80186E393E00E94B7162D
:100B4000C82F811133C0B8018EED92E00E940B11C5
:100B5000C82F81112BC0B80180EE92E00E94611372
:100B6000C82F811123C04EEF52E0B80186E493E014
:100B70000E94021981111AC066EF72E0C8010E943A
:100B80001A30892B99F46CEE72E08BEE93E00E94A0
:100B90001F2784E690E00E946D0460E28BEE93E0F4
:100BA0000E94432784E690E00E946D048C2FCF9131
:100BB0001F910F91089580E00895BC0185E293E0B4
:100BC0000C94CE14CF93DF93EC01BC0182E191E051
:100BD0000E94931EBE0187E693E00E94FB1A80E00C
:100BE000DF91CF91089586E493E00E9447198CE746
:100BF00093E00E94632282EB93E00E94D12382E182
:100C000091E00E94041E87E693E00E94B31A80E000
:100C100008958091590190915A010E94CA0A86E074
:100C20000E94D91781E08093B20360E071E080EE0A
:100C300092E00E94481380913B038F770C94E40B61
:100C40008091590190915A010C94830B1092B50137
:100C5000089588E492E00E948B0E87E892E00E945B
:100C6000251089E692E00E94390F8FEC92E00C94F7
:100C70007210EBE5F1E050E040E070E060E0000071
:100C80009191A92FB0E084E0B595A7958A95E1F7F9
:100C900090962C9130E09F7002C0359527959A95DB
:100CA000E2F72095309521703327042E02C0220FE1
:100CB000331F0A94E2F7622B732B4F5F5F4F4C3068
:100CC0005105E9F6CB0108951F93CF93DF93C8E157
:100CD000D2E010E0288139818A819B81482F440F1E
:100CE0004270522F5170452B09F005C1AC01569549
:100CF0004795440F427021FB552750F9452B09F0C9
:100D0000EFC0AC015695479556954795440F4270F4
:100D100022FB552750F9452B09F0D7C0AC01569559
:100D200047955695479556954795440F427023FB36
:100D3000552750F9452B09F0BDC0AC01529542959D
:100D40004F7045275F704527440F427024FB55279D
:100D500050F9452B09F0A3C0AC0156954795529523
:100D600042954F7045275F704527440F427025FB21
:100D7000552750F9452B09F087C0AC010024440FDA
:100D8000551F001C440F551F001C452F502D440FAC
:100D9000427026FB552750F9452B09F06AC0AC017B
:100DA000440F452F441F550B5195440F427027FBAC
:100DB000222720F9422B09F052C0492F440F4270DC
:100DC000232F2170422B09F040C031FB222720F94C
:100DD000492F4270422B79F5492F4695427032FBDC
:100DE000222720F9422BE9F4292F269526952270F7
:100DF00033FB442740F9422B59F4998388832A9680
:100E0000145F103309F066CFDF91CF911F910895E1
:100E10006BE0610F80E090E00E94D70C8A819B819B
:100E2000ECCF6AE0610F80E090E00E94D70C39813E
:100E30008A819B81D9CF69E0610F80E090E00E94B8
:100E4000D70C39818A819B81C7CF68E0610F80E030
:100E500090E00E94D70C39818A819B81B6CF67E0F0
:100E6000610F80E090E00E94D70C39818A819B81DC
:100E7000A4CF66E0610F80E090E00E94D70C28814B
:100E800039818A819B818BCF65E0610F80E090E0A2
:100E90000E94D70C288139818A819B816ECF64E0C2
:100EA000610F80E090E00E94D70C288139818A810F
:100EB0009B8152CF63E0610F80E090E00E94D70CED
:100EC000288139818A819B8138CF62E0610F80E07F
:100ED00090E00E94D70C288139818A819B811ECFA6
:100EE00061E0610F80E090E00E94D70C2881398199
:100EF0008A819B8106CF612F80E090E00E94D70C11
:100F0000288139818A819B81F1CE88E492E00E9418
:100F1000E60D811104C088E492E00C94E90D87E8A5
:100F200092E00E946B0F89E692E00C94130F88E424
:100F300092E00E94E60D811104C088E492E00C94D6
:100F4000840E87E892E00E941F1089E692E00C94DC
:100F5000000FCF93C82F88E492E00E94E60D6C2F1B
:100F6000811105C088E492E0CF910C94250E87E8AA
:100F700092E0CF910C94CF0FCF93C82F83FF03C083
:100F800081EE0E94A907C0FF03C080EE0E94A9075E
:100F9000C1FF03C082EE0E94A907C2FF03C086EE14
:100FA0000E94A907C4FF04C083EECF910C94A90747
:100FB000CF910895CF93C82F892F0E94BC078C2F03
:100FC000CF910C94A907CF93C82F88E492E00E9498
:100FD000E60D6C2F811105C088E492E0CF910C944E
:100FE0004C0E87E892E0CF910C94F60FFC019081B3
:100FF000DB018C91981305C081E0218111969C91B1
:10100000291380E008951F93CF93DF9300D000D081
:10101000CDB7DEB7182F803368F5E82FF0E0EE0F7C
:10102000FF1FED5AFB4F808191819C838B838FEF53
:1010300089838A83BE016F5F7F4FCE0103960E9432
:10104000F607882369F0A12FB0E0A454BE4FE091C9
:101050000201F0910301612F8C9109958B839C8390
:101060008B819C810F900F900F900F90DF91CF910B
:101070001F9108951092B3041092B404E3EBF4E0CE
:10108000D2CF1F93CF93DF93C62F172F862F972F83
:101090000E947A05823009F1812F807C61F480E220
:1010A0008C0F883008F010E08C2F912FDF91CF91BA
:1010B0001F910C94DA07812F887C883471F4612F9A
:1010C00070E0762F66276C0F711D737089E692E0D1
:1010D000DF91CF911F910C94EB0EDF91CF911F9177
:1010E00008958F929F92BF92CF92DF92EF92FF92DC
:1010F0000F931F93CF93DF9300D000D000D0CDB7D4
:10110000DEB77C016B010E94970710E000E0BB2472
:10111000BA940033110599F1F6019081901729F1E5
:10112000003330F5F801EE0FFF1FED5AFB4F8080C2
:1011300091809E828D82BB82BC82BE016D5F7F4F9B
:10114000CE0105960E94F60781110FC019821A82FE
:10115000BE016F5F7F4FCE0105960E94F607811199
:1011600004C0B401C7010E9441080F5F1F4FD1CFD7
:101170001092B3041092B404E3EBF4E0D8CF2696B7
:101180000FB6F894DEBF0FBECDBFDF91CF911F9198
:101190000F91FF90EF90DF90CF90BF909F908F9036
:1011A0000895EF92FF920F931F93CF93DF938C01DB
:1011B000EB01898181FF43C080FD41C08B81807C30
:1011C000F1F5888180930101FA8088E492E00E9421
:1011D000E60D6F2D81112EC088E492E00E94950EDD
:1011E000882301F1FB80EA80F3FE03C081EE0E94B8
:1011F000E307F0FE03C080EE0E94E307F1FE03C0A8
:1012000082EE0E94E307F2FE03C086EE0E94E3072F
:10121000F4FE03C083EE0E94E3078E2D0E94E307D5
:101220000E9485078B81882379F00E94BC070E9469
:1012300085070AC087E892E00E94B90FD1CFE091FC
:1012400001018881E81317C0898181FF07C080FDF3
:1012500005C06A817B81C8010E944108CE010E94BD
:10126000DD058230E9F0DF91CF911F910F91FF9062
:10127000EF900C948507E03360F4F0E0EE0FFF1F71
:10128000ED5AFB4F8181982F907CF1F60E94BC07AC
:10129000DBCF1092B3041092B404E3EBF4E0F2CF8E
:1012A000DF91CF911F910F91FF90EF900895FF92E2
:1012B0000F931F93CF93DF93CDB7DEB72D970FB664
:1012C000F894DEBF0FBECDBF8C0129873A874B87CC
:1012D0005C876D87203348F430FF61C031FD5FC00B
:1012E00089850E9403089C878B87CE0109960E94FE
:1012F0002705823009F447C0E985E03368F49A8510
:10130000F0E0EE0FFF1FED5AFB4F90FF55C091FD2F
:1013100053C09FEF90839183811135C01F8218863F
:10132000BE01695F7F4FCE010B960E94F6078111C7
:101330002AC01D821E82BE016B5F7F4FCE010B96BD
:101340000E94F60781111FC0FF24FA94FB82FC82E1
:10135000BE016D5F7F4FCE010B960E94F607811193
:1013600012C0F982FA82BE016F5F7F4FCE010B96E9
:101370000E94F607811107C08C85843409F5CE01DF
:1013800009960E94750C2D960FB6F894DEBF0FBE1D
:10139000CDBFDF91CF911F910F91FF9008958FEFF7
:1013A00089838A83BE016F5F7F4FCE010B960E94B7
:1013B000F607811195CF99CF9C852B852083ABCFE4
:1013C0008F7C8134B9F48A851B8581FF0AC080FD3A
:1013D00008C0612F8FEC92E00E94761010931002EB
:1013E000D2CF809110028113CECF8FEC92E00E9479
:1013F0007410C9CFBE01675F7F4FC8010E9471089A
:10140000BE01675F7F4FC8010E94D108CE010996D7
:101410000E94E205B8CFEF92FF920F931F93CF93F4
:10142000DF9300D000D000D01F92CDB7DEB7022FDF
:101430002B833C834D835E836F83203308F042C04F
:101440007C01832F817031FF22C081113BC08FEF5F
:1014500089838A83BE016F5F7F4FCE0105960E940C
:10146000F607882329F0802F0E9403089E838D832E
:10147000CE0103960E941305811124C02B813C816B
:101480004D815E816F81C7010E9457091BC088236F
:10149000C9F010E0000F111F0D5A1B4FF801808199
:1014A00091819E838D8319821A82BE016F5F7F4F67
:1014B000CE0105960E94F6078823D1F28FEFF8013E
:1014C0008083818327960FB6F894DEBF0FBECDBF11
:1014D000DF91CF911F910F91FF90EF900895CF93DF
:1014E0000FB6F894A89580916000886180936000A1
:1014F000109260000FBEABE5B1E047E651E061E05D
:1015000070E08D91E82FF0E024E0F595E7952A95BD
:10151000E1F7C1A18F709B0101C0220F8A95EAF704
:10152000922F90959C2391A382A1822B82A34A178C
:101530005B0739F7A7E6B1E04BE651E061E070E008
:101540008D91E82FF0E094E0F595E7959A95E1F715
:1015500091A18F709B0101C0220F8A95EAF7922B0F
:1015600091A382A1822B82A34A175B0749F780E1EE
:10157000809381001092800080EE9EE2909387001D
:101580008093860081E18093810081E080936F00E9
:10159000CF91089585B7806885BF85B7806885BF7E
:1015A0000E94290683E192E00E946F0A40E855E21A
:1015B00060E070E08BEE93E00E9419260E94CE045A
:1015C0000E94FB04E3E5F4E081E39FEF815021F00A
:1015D000908391833296FACF8BEB91E00C94E20BDF
:1015E0006F927F928F929F92AF92BF92CF92DF9233
:1015F000EF92FF920F931F93CF93DF9327E6E22E94
:1016000021E0F22EC8E1D2E03BE6632E31E0732EFA
:10161000912C812CAA24A394B12CF70181917F01F4
:10162000082F10E0159507951595079515950795C1
:1016300015950795F80192A18F70650101C0CC0C3A
:101640008A95EAF7892F8C2582A30E943906F80132
:1016500022A1C226C2A248855985842795276C817C
:101660007D812E813F8126273727282339233F83F9
:101670002E83FB01E095F095E823F923FD83EC83AD
:101680008623972320953095822393234827592733
:1016900059874887882A992A8114910401F18091F9
:1016A00020029091210290931B0280931A02809154
:1016B0002A0290912B02909325028093240280911C
:1016C00034029091350290932F0280932E028091E4
:1016D0003E0290913F0290933902809338022A96FD
:1016E0006E147F0409F099CFDF91CF911F910F9174
:1016F000FF90EF90DF90CF90BF90AF909F908F9032
:101700007F906F9008950E9403046093B7017093D7
:10171000B8018093B9019093BA010E940D058091A0
:101720001302882331F01092130283E192E00E94A9
:10173000F00A0E9464060C94F30570E090E3899F20
:10174000600D711D1124660F771FFB01E455FF4FDB
:101750008491FB01E355FF4F94910895EF92FF921E
:101760000F931F93CF93DF93ECEBF1E080E3DF0166
:101770001D928A95E9F77F0110E01033E1F0C091E6
:101780000401D0E0C451DE4FB1E0CC3EDB0771F084
:101790000A91E0910201F0910301612F802F0995D8
:1017A0008F3F11F49F3F81F3F70100831F5FFFEF2D
:1017B000EF1AFF0AE2CFDF91CF911F910F91FF90B7
:1017C000EF9008950C94AE0B90910001891708F0EA
:1017D00080E091E0909304018093EC010E94AE0BB5
:1017E0000C94DB054091040150E090E0682F70E01C
:1017F000292F092E000C330B2417350764F42451CC
:101800003E4FF9012081022E000C330B26173707BB
:1018100021F09F5FEDCF80E0089581E00895CF93A0
:10182000909100018917A0F4C82F0E94F20B81113A
:101830000FC0E091040181E08E0F80930401F0E07D
:10184000E451FE4FC0830E94AE0BCF910C94DB0598
:10185000CF910895CF93DF93D82F0E94F20B882366
:1018600081F1C0910401C23028F480E0DF91CF9172
:101870000C94E40BECEEF1E090E080E02D2F30E0F2
:101880004191042E000C550BBC016F5F7F4F421736
:10189000530799F44C2F50E0481B590B64517E4F6D
:1018A00084519E4F0E944730C150C09304010E9452
:1018B000AE0BDF91CF910C94DB05CB016C1700F3DD
:1018C000F6CFDF91CF910895E0910401F0E0E5516A
:1018D000FE4F80818F5F0C940F0CE0910401F0E0CB
:1018E000E551FE4F80810C942A0CCF93DF93FC01CD
:1018F000C2819181292F2270C43558F0222309F426
:1019000050C090FD4EC08CEA8C0FDF91CF910C94AB
:10191000E40BCA32C8F1D6EDDC0FD13251F0D2322D
:1019200081F4222351F090FD08C0DF91CF910C94F7
:10193000640C2223D1F390FDF8CFDF91CF910C946A
:101940006D0C211110C0A3E5B4E081E38150B9F022
:101950009C91C91306C011962C9111979381291758
:1019600001F11296F3CF90FDEECF8D2F0E94F20B76
:10197000811117C08D2FDF91CF910C940F0C8D2FFB
:10198000DF91CF910C942A0C222359F090FD09C0CD
:101990008C2F0E94F20B882311F08C2FF1CF8C2F0B
:1019A000EACFDF91CF910895109210020895CF935E
:1019B000DF9300D000D01F92CDB7DEB7262F342F93
:1019C000842F817041FF15C0811115C08091520490
:1019D00061E0680F609352044FEF5FEF86EB91E098
:1019E0000F900F900F900F900F90DF91CF910C946C
:1019F0000B0A8111EBCF0F900F900F900F900F906B
:101A0000DF91CF9108951F920F920FB60F9211247C
:101A10008F9381E0809313028F910F900FBE0F90F0
:101A20001F901895FC0182818F5BFB01808381E010
:101A30000895CF93DF93CDB7DEB769970FB6F894CB
:101A4000DEBF0FBECDBFFC01DB019C919F5F9C936D
:101A50009E012D5F3F4F81E1D9011D928A95E9F7E3
:101A600029E0298384E08A8391E09D8383E08E834B
:101A70009F8398872A8721E22B879C879D879F8752
:101A800022E2288B2FE3298B27E02B8B25E02C8B60
:101A90008E8B20E430E0388F2F8B998F82818B835F
:101AA000838180688D8B49E150E0BE016F5F7F4F7D
:101AB00080E00E94632A69960FB6F894DEBF0FBEDD
:101AC000CDBFDF91CF910895FC01DB018C9181386E
:101AD000A9F413968C911397823281F42281149683
:101AE0008D919C912817190649F48285848F4FE3C4
:101AF00050E066E073E080E80C94632A90E080E0B8
:101B00000895FC01DB01228114968D919C9115971B
:101B10002817190681F511968C9111979C91913A8D
:101B200069F4813029F0833029F4848D8093F100A9
:101B300081E008958230F9F4858DF8CF9132D9F49F
:101B40008B3021F412968C91848FF2CF8A3011F46D
:101B5000158EEECF893079F4CF0116962D913C91F8
:101B6000179713964C91423041F461E070E04E9625
:101B70002130310551F080E008954130E1F72830FF
:101B80003105C9F768E070E00B960E94892AD0CF32
:101B9000CF93DF93EC0181E08C838D839E01255EE2
:101BA0003F4F3F832E83198618862FE631E0398315
:101BB00028836A876C8F8D8F1E8E81EC8B8F0E949D
:101BC000FC26BE01DF91CF910C94B826FC01848DD8
:101BD0000895EF92FF920F931F93CF93DF938C01A1
:101BE000EC012B967C0183E1E80EF11C48E050E00B
:101BF000BE01C7010E943130892B21F1F801838198
:101C000048E050E0BE0180640E94B2298C01E0915E
:101C10006702F0916802309731F09C0148E050E093
:101C2000BE0182E0099588E0FE01D70101900D9286
:101C30008A95E1F7C801DF91CF911F910F91FF9035
:101C4000EF9008950FEF1FEFF5CFFC0180E2860FB4
:101C5000883070F4605E770B21E030E001C0220F25
:101C60006A95EAF78385822B838781E090E0089567
:101C7000DF011D9690E080E02D912617B1F3211130
:101C800004C0E80FF91F6587F0CF019686309105F3
:101C900099F790E080E00895CF93DF9320E2260F3C
:101CA000283090F4605E770B21E030E001C0220F15
:101CB0006A95EAF72095FC0133852323238781E089
:101CC00090E0DF91CF910895DC011D969C012D5E7F
:101CD0003F4FFD014191461303C0EF012197188248
:101CE000E217F307B9F720E03D91332349F0EC0107
:101CF000C20FD11D4D853D87ED01219748832F5F90
:101D0000AE17BF0789F7DBCF0B9628E0FC011192D5
:101D10002A95E9F70895CF93DF93EC010E94840E92
:101D2000CE01DF91CF910C94E90DFC013D964396D5
:101D30002191261729F0E817F907D1F780E00895D7
:101D400081E0089520914002309141024091420289
:101D50005091430260914402709145028091460285
:101D600090914702A1E00E94F92F20934002309306
:101D700041024093420250934302609344027093A5
:101D8000450280934602909347020E94053029F451
:101D900061E088E492E00C94C80D08958091790286
:101DA000811113C0109282021092810285E493E0A7
:101DB000909384028093830289E190E0909386025D
:101DC0008093850281E0809379020E94362E61E83B
:101DD00072E00C94A32DFC0130E020E04191519180
:101DE000452B41F4220F331F280F391FF90171834E
:101DF000608308952F5F3F4F2430310579F70895B0
:101E000028E0FC0111922A95E9F70895CF93DF931A
:101E1000EC010E94362E28E030E0AE0164E0DF9154
:101E2000CF910C94F32D0F931F93CF93DF93EC017D
:101E30008C01085F1F4F48E050E0BC01C8010E94C0
:101E40003130892B51F0CE010E94060F88E0FE014F
:101E5000D80101900D928A95E1F7DF91CF911F9102
:101E60000F91089528E0FC0111922A95E9F70C944E
:101E7000130F0C94320F89E692E00C94CE0E8091F1
:101E8000C102811113C01092CA021092C9028EE5DC
:101E900093E09093CC028093CB0281E490E0909306
:101EA000CE028093CD0281E08093C1020E94362E43
:101EB00069EC72E00C94A32DCF93DF93EC010E94A8
:101EC000362EAE01435E5F4F2DE130E068E0DF91DA
:101ED000CF910C94F32DEF92FF920F931F93CF931A
:101EE000DF93EC01F8808D8D8E010F5F1F4F8F15F2
:101EF000D9F0F801AE01435E5F4F20E0858D30815F
:101F00003196932F9095982319F08323848F21E0A5
:101F1000E417F50799F7222319F0CE010E945C0F10
:101F2000FD8ECE010E945C0F7E018EE1E80EF11C59
:101F30004CE150E0B801C7010E943130892B81F09B
:101F40008CE1F801D70101900D928A95E1F7CE015D
:101F5000DF91CF911F910F91FF90EF900C945C0F48
:101F60008FEF9FEFDF91CF911F910F91FF90EF9037
:101F700008956E3D90F4E62FE695E695E695E80F18
:101F8000F92FF11D677021E030E001C0220F6A9542
:101F9000EAF79181922381E009F480E008956E3D93
:101FA000A0F4E62FE695E695E695E80FF92FF11DEA
:101FB000677021E030E001C0220F6A95EAF7818165
:101FC000822B818381E090E00895605E683058F450
:101FD00041E050E001C0440F6A95EAF7FC0120811E
:101FE000242B2083EFCF90E080E008956E3DA8F48D
:101FF000E62FE695E695E695E80FF92FF11D677057
:1020000021E030E001C0220F6A95EAF72095818136
:102010002823218381E090E00895605E683060F4B9
:1020200021E030E001C0220F6A95EAF72095FC011B
:10203000308123232083EECF90E080E008952DE1CE
:10204000FC0111922A95E9F70895CF93DF93EC01F3
:102050000E941F10CE01DF91CF910C945C0F87E896
:1020600092E00C943F0F8091D002811113C0109226
:10207000D9021092D8028FE993E09093DB0280930B
:10208000DA0288E190E09093DD028093DC0281E047
:102090008093D0020E94362E68ED72E00C94A32D3E
:1020A0000F931F93CF93DF93EB018A010E94362E8B
:1020B0009801AE0165E0DF91CF911F910F910C94D3
:1020C000F32DCF93DF931F92CDB7DEB7198241E096
:1020D00050E0BE016F5F7F4F0E9450100F90DF9164
:1020E000CF9108950C9461100C946110CF93DF93FD
:1020F0001F92CDB7DEB76983633841F488E494E07A
:102100000E949C2C0F90DF91CF91089541E050E008
:10211000BE016F5F7F4F0E945010F4CF8FEC92E0B2
:102120000C943310FF920F931F93CF93DF93EC0126
:102130008B01FB01F0800E945930F81621F06F2DC1
:10214000CE010E946130F801F1802196CE010E94FB
:102150005930F81621F06F2DCE010E946130C80170
:10216000DF91CF911F910F91FF900895CF92DF9251
:10217000EF92FF920F931F93CF93DF937C0162E066
:1021800070E087E393E00E946815EC01F70191830A
:1021900080838C016C01F2E0CF0ED11C0C151D0563
:1021A00040F4C8010E9459308F3F41F40F5F1F4F28
:1021B000F5CF65E071E0CE010E949210F701C08179
:1021C000D181CE010E94593080930501CE01019644
:1021D0000E9459308093060180E0DF91CF911F91DA
:1021E0000F91FF90EF90DF90CF9008956BEE73E02A
:1021F0008BEE93E00E941F2784E690E00E946D041E
:102200006AE08BEE93E00E94432784E690E00E9410
:102210006D0480E008950F931F93CF93DF93EC013B
:102220008B0141ED53E086E493E00E940219811195
:1022300044C067EB73E0C8010E941A30892BE9F5AE
:102240008BEE93E00E942B258A309105C9F0019610
:10225000B9F041E070E060E08BEE93E00E942E2840
:10226000609305017093060165E071E088819981B2
:102270000E94921081E0DF91CF911F910F910895FC
:102280006091060170E0762F662780910501680F46
:10229000711D4AE050E08BEE93E00E94C02784E677
:1022A00090E00E946D0460E28BEE93E00E94432771
:1022B00084E690E00E946D04D7CF80E0DCCFCF931E
:1022C000DF93DC01EB019A818C91981305C02B817F
:1022D00011968C91281749F09E3721F080E0DF910C
:1022E000CF9108958B81813DC9F7898181FFF6CF18
:1022F00080FDF4CF87FDF2CF82E191E00E94FD1CCA
:10230000882361F361E082E191E00E94611D1A82FD
:102310001B8281E0E4CF0C9459308F929F92AF9250
:10232000BF92CF92DF92EF92FF920F931F93CF93C2
:10233000DF938C01FC01E080F18015821482C28061
:10234000D380CE0CDF1C4701B12C8C149D0408F007
:102350004BC0E4012196C4010E948B118E3008F01D
:1023600043C0E82FF0E0E954FE4E0C94D92FE6115B
:10237000C511C511C911C911C911C511C511C511A1
:10238000C711C711C711CC11DB11E40122964E0110
:10239000DCCFE4012396FBCF4E01CE010E948B11CE
:1023A000A82E2296C40101960E948B11A110F4CF91
:1023B0008111F2CFECCF2C2F9D2F2196822F0E94DE
:1023C0008B112C2F9D2F8111F8CFE1CFB394EB2DE2
:1023D000F0E03296EE0FFF1FE00FF11FCE018E19D5
:1023E0009F0991838083D3CF8B2DDF91CF911F9154
:1023F0000F91FF90EF90DF90CF90BF90AF909F90A4
:102400008F9008958F929F92AF92BF92CF92DF925A
:10241000EF92FF920F931F93CF93DF93FC01EC5B3E
:10242000FF4F2081621708F0DFC07C01E62FF0E04B
:102430003296EE0FFF1FEE0DFF1DD7010D911C917F
:1024400080819181080F191FD12CF7018081918122
:1024500022813381820F931F0817190708F0C4C027
:10246000E8012196C8010E948B1181508D3008F03F
:10247000BBC0E82FF0E0E15CFD4E0C94D92F6B124D
:102480007A1286129712A812B912C512D1127212BC
:10249000721272124C12DD128D2C912CB12CA12CC7
:1024A000CE010E948B11C82E8E010E5F1F4FCE01F0
:1024B00001960E948B11811102C0CC2091F0682FEF
:1024C0007C2D85E293E00E94A914C501B4010E940D
:1024D0003404E801E5CF0E5F1F4FCE010E948B113F
:1024E000D82EE8016D2D70E090E080E00E94340469
:1024F0008E01ABCF0E5F1F4FCE010E948B11682F54
:1025000070E090E080E00E943404EBCFCE010E94A6
:102510008B11C82EE8012396C80102960E948B11E8
:10252000682F7C2D85E293E00E940514DBCFCE015D
:102530000E948B11C82EE8012396C80102960E94C2
:102540008B11682F7C2D85E293E00E944014CACF46
:10255000CE010E948B11C82EE8012396C801029675
:102560000E948B11682F7C2D85E293E00E94A914B4
:10257000B9CF0E5F1F4FCE010E948B11682F70E004
:1025800085E293E00E940514ACCF0E5F1F4FCE0191
:102590000E948B11682F70E085E293E00E94401446
:1025A000A0CF0E5F1F4FCE010E948B11682F70E0ED
:1025B00085E293E00E94A91494CFCE018D2C912C3A
:1025C000B12CA12C21960E948B11882309F48ACF6B
:1025D000682F70E085E293E00E94A914C501B40160
:1025E0000E943404CE01EECFDF91CF911F910F9165
:1025F000FF90EF90DF90CF90BF90AF909F908F9023
:102600000895292F30E0322F222790E08C55914DEC
:10261000280F391F81E02032310508F080E008954D
:102620000F931F93CF93DF938C01EB018A819B81E2
:102630000E9401138823A9F0898181FF0DC080FDCC
:102640000BC06A816C55C8010E94021281E0DF91C3
:10265000CF911F910F91089585E293E00E94681435
:10266000F5CF80E0F4CF67E274E08BEE93E00E9458
:102670001F2784E690E00E946D046AE08BEE93E0F1
:102680000E94432784E690E00E946D0480E0089554
:102690000F931F93CF93DF93EC018B0187E393E0BC
:1026A0000E946815998388831B830A83CE010E9448
:1026B0008D11CC5BDF4F8883DF91CF911F910F91FC
:1026C0000895BF92CF92DF92EF92FF920F931F93E4
:1026D000CF93DF93EC018B014DE054E086E493E06F
:1026E0000E940219811186C047E050E065E074E065
:1026F000C8010E942330892B09F07CC0095F1F4F5D
:1027000061E074E0C8010E941A30892B09F05FC0B3
:102710008BEE93E00E942B25F12CE12C8A30910561
:1027200011F0019621F58A819B81E816F90608F0DF
:102730004EC0888199818E0D9F1D0E948B114AE0A9
:1027400050E0682F8BEE93E00E94B92784E690E07A
:102750000E946D0460E28BEE93E00E94432784E6C2
:1027600090E00E946D048FEFE81AF80ADCCF8BEE40
:1027700093E00E942B258A30910511F1019601F119
:102780008A819B81E816F906D8F441E070E060E0A8
:102790008BEE93E00E942E28B62E67018FEFC81AA9
:1027A000D80A88819981E80EF91EC7010E94593024
:1027B000B81621F06B2DC7010E9461307601D7CF8A
:1027C000CE010E948D11FE01EC5BFF4F808369EF0B
:1027D00073E0C8010E941A30892B51F441E070E087
:1027E00060E08BEE93E00E942E28CE010E94021240
:1027F00081E001C080E0DF91CF911F910F91FF90A8
:10280000EF90DF90CF90BF900895EF92FF920F93DB
:102810001F93CF93DF9300D000D01F92CDB7DEB7C8
:102820008C01F62EE72E609152048FEF898382E8A7
:102830008A83FB827C836D832FEF32E84F2D572FE5
:1028400086EB91E00E945709C8014096F801E8170D
:10285000F90741F02081211111C0218121110EC001
:10286000F082E1820F900F900F900F900F90DF9108
:10287000CF911F910F91FF90EF9008953296E7CF7F
:10288000CF93DF9300D000D01F92CDB7DEB7AB015E
:102890009C01205F3F4FFC012E173F0751F08081C4
:1028A000841305C08181851302C010821182329683
:1028B000F3CF609152042FEF31E886EB91E00F9057
:1028C0000F900F900F900F90DF91CF910C945709BC
:1028D000CF92DF92EF92FF920F931F93CF93DF93EC
:1028E00000D000D01F92CDB7DEB77C0120E1E20E10
:1028F000F11C8C01DD24DA9481E8C82EE016F10683
:10290000D1F0F80140815181411102C0552381F07D
:1029100060915204D982CA824B835C836D832FEF0E
:1029200031E886EB91E00E945709F801108211828C
:102930000E5F1F4FE3CF0F900F900F900F900F90EF
:10294000DF91CF911F910F91FF90EF90DF90CF908B
:1029500008950F931F93CF93DF9300D000D01F9261
:10296000CDB7DEB78B01609152042FEF32E8A8019A
:1029700086EB91E00E945709609152042FEF31E8F5
:10298000A80186EB91E00F900F900F900F900F90A1
:10299000DF91CF911F910F910C9457090F931F93C3
:1029A000CF93DF938C01005F1F4FEC010C171D07C5
:1029B00071F06881798189819881911102C08823A1
:1029C00021F086EB91E00E9441082296EFCF80E053
:1029D000DF91CF911F910F91089584E690E00C94C0
:1029E0006D044AE050E0682F8BEE93E00E94B92717
:1029F0000E94ED1460E28BEE93E00E9443270C945A
:102A0000ED14FF920F931F93CF93DF93EC01F62EFB
:102A100008811981C8010E945930F81621F06F2DE4
:102A2000C8010E946130CE01DF91CF911F910F91BB
:102A3000FF900895AF92BF92CF92DF92EF92FF92F4
:102A40000F931F93CF93DF9300D0CDB7DEB78C01E8
:102A50006C0184E0C80ED11C5601F12CE12CC70199
:102A60000E945930F50181935F01FFEFEF1AFF0AD1
:102A700084E0E816F10499F7F80185818F3FD1F4DD
:102A80008481982F9F779F3711F487FD148281E00E
:102A9000F801858310E000E01A830983F601619153
:102AA0006F01CE0101960E9401150F5F1F4F043088
:102AB000110591F780E00F900F90DF91CF911F915A
:102AC0000F91FF90EF90DF90CF90BF90AF9008955F
:102AD0000F931F93CF93DF9300D0CDB7DEB77A83E8
:102AE0006983FC01238110E000E021110FC0008107
:102AF0001181CB01800F911F9183808342E0BE0141
:102B00006F5F7F4F8FE393E00E945717C8010F90CC
:102B10000F90DF91CF911F910F910895CF92DF9287
:102B2000EF92FF920F931F93CF93DF9300D0CDB717
:102B3000DEB77C016C0184E0C80ED11C10E000E01F
:102B40001A830983F60161916F01CE0101960E94FB
:102B500001150F5F1F4F0430110591F781E0F70158
:102B600082830F900F90DF91CF911F910F91FF9073
:102B7000EF90DF90CF9008951F93CF93DF93EC01F8
:102B8000162F80910001681748F4862F0E94E40BED
:102B90008C818078912F9F77892B8C831E3720F032
:102BA0008C8180788E678C83CE010E948E158C81FB
:102BB0008F77DF91CF911F910895FC01948160FB85
:102BC00097F99483892F8F778F3719F490789E67C0
:102BD0009483CF010C948E15CF93DF93EC0181E0A9
:102BE0008B8360E18FE393E00E943E178D818130FB
:102BF00021F01A82DF91CF9108952E813F8180913B
:102C00003F03909140032F3F320769F49F838E83E7
:102C1000CE010E948E158C818F778E3758F7DF9109
:102C2000CF910C94E40B2817390721F7F4CFFC015E
:102C30002381211102C00E94EC1580E0089584E0F8
:102C400090E0909338038093370308958BEE93E0E0
:102C50000E942B259C0181E02A30310529F02F3F6D
:102C60003F4F11F080E0089508950F931F93CF9385
:102C7000DF9300D0CDB7DEB78B014EE554E086E49C
:102C800093E00E940219811135C06EE474E0C8011E
:102C90000E941A30892BF1F40E94261610E000E001
:102CA000811149C00E94261681113DC041E070E0AB
:102CB00060E08BEE93E00E942E281A830983CE01F8
:102CC00001960E9401150F5F1F4F011584E0180740
:102CD00049F729C062E474E0C8010E941A30892BC8
:102CE00059F065E374E0C8010E941A3010E000E07A
:102CF000892B69F180E018C08091370390913803E7
:102D000060E074E0681B790B4AE050E08BEE93E0E2
:102D10000E94C0270E94ED1460E28BEE93E00E94B7
:102D200043270E94ED1481E00F900F90DF91CF9127
:102D30001F910F910895C8010E9459300E94F1140B
:102D40000F5F1F4F011584E01807A9F7ECCF1A8316
:102D500009836FEFCE0101960E9401150F5F1F4F8F
:102D6000011584E0180799F70E94BE2CDCCFCF93A1
:102D7000DF93EB0143EB54E086E493E00E940219F9
:102D800081117AC049E050E069EA74E0CE010E9406
:102D90002330892B09F070C029966CE974E0CE01CC
:102DA0000E941A30892B81F40E942616811160C07E
:102DB00041E070E060E08BEE93E00E942E2887E314
:102DC00093E00E94BC1540C065E974E0CE010E940A
:102DD0001A30892BE9F16DE874E0CE010E941A30B7
:102DE000892B71F169E874E0CE010E941A30892BB9
:102DF00009F042C080913A03D0E0C0E0882321F07E
:102E0000C0913D03D0913E0360913F037091400318
:102E10004AE050E08BEE93E00E94C0270E94ED1440
:102E200067E874E08BEE93E00E941F270E94ED1488
:102E30004AE050E0BE018BEE93E00E94C02715C02F
:102E400080913C030E94F11481E0DF91CF910895BD
:102E50006091390386E493E00E9439190E94ED14D1
:102E600060E28BEE93E00E9443270E94ED14ECCFCA
:102E700080913B038F77E6CF80E0E7CFFC01208194
:102E800031812170332781E0861770F440815181B0
:102E90005695479551834083220F331F4170552724
:102EA000242B352B8F5FF0CF318320830895DC01F5
:102EB000FB01415000F181912D913C91119768E007
:102EC00070E051E0982F952399F4932F991F99273B
:102ED000991F220F331F992319F095E029273058A5
:102EE000550F6150710971F711963C932E93E1CF04
:102EF000932F9095EBCF089584E690E00C946D04A9
:102F00001F93CF93DF9390914303891730F080E0B4
:102F100090E0DF91CF911F910895C62FD0E090E30C
:102F2000899FC00DD11D1124CC0FDD1F609144037A
:102F300070914503C60FD71FCE010E945930182F3C
:102F4000CE0101960E945930912FE3CF9091420318
:102F5000891710F40C949D0B891B0C94801787E340
:102F600093E00E941A15809100018093420380E053
:102F7000089568E475E08BEE93E00E941F270E949D
:102F80007C176AE08BEE93E00E9443270E947C1737
:102F900080E008958093430390E6899FB001112457
:102FA00087E393E00E946815909345038093440360
:102FB00008958093000190913B0320E837E197FD4D
:102FC00007C090914203980F9093000126EA37E1E1
:102FD00030930301209302010C94CA17FF920F93C0
:102FE0001F93CF93DF9300D0CDB7DEB7F62E672FB8
:102FF0008C01000F111F8091440390914503800FB5
:10300000911F9A838983CE0101960E9401158091B8
:103010004403909145030196800F911F9A83898301
:103020006F2DCE0101960E9401150F900F90DF9138
:10303000CF911F910F91FF900895FF920F931F93CF
:10304000CF93DF93F82E8B01C0E0CF15F9F0D0E0DD
:103050006D2F8C2FF8010995692F70E0762F662768
:10306000680F711D4AE050E08BEE93E00E94C0278C
:103070000E947C1760E28BEE93E00E9443270E943F
:103080007C17DF5FD03321F7CF5FDFCFDF91CF91A8
:103090001F910F91FF9008958BEE93E00E942B25D6
:1030A0009C0181E02A30310529F02F3F3F4F11F07C
:1030B00080E008950895FF920F931F93CF93DF93BD
:1030C0001F92CDB7DEB78B0149E155E086E493E06E
:1030D0000E94021981118EC047E050E061E175E065
:1030E000C8010E942330892B09F084C0095F1F4F5B
:1030F00066E075E0C8010E941A30892BE1F50E9454
:103100004C188823B1F060913B0367FB662760F998
:103110004AE050E08BEE93E00E94B9270E947C17B2
:1031200060E28BEE93E00E9443270E947C1781E0CF
:1031300062C041E070E060E08BEE93E00E942E28D8
:10314000162F698387E393E00E94DD159091430376
:1031500090930001112339F080E897E190930301E7
:1031600080930201E4CF80914203890F8093000194
:1031700086EA97E1F3CF6EEF74E0C8010E941A303F
:10318000892B39F46DE97BE0809142030E941D1880
:10319000CECF67EF74E0C8010E941A30892B51F539
:1031A0000E944C1810E000E090E3F92E882329F0EB
:1031B00060E877E180914303E9CF0E944C188111C8
:1031C000B6CF809143038F9DC001112408171907C2
:1031D00008F0ADCF41E070E060E08BEE93E00E943C
:1031E0002E28272F3327722FC8010E94EE170F5F5A
:1031F0001F4FE3CF80E00F90DF91CF911F910F9190
:10320000FF900895CF93DF93CB01EA016FE875E05B
:103210000E941A30892B49F4BE018BEE93E00E9484
:103220004E2781E0DF91CF91089580E0FBCFCF93CF
:10323000DF93EB0145E755E00E940219811117C0A9
:1032400068E675E0CE010E941A30892B31F40E94A5
:10325000BE2C81E0DF91CF91089560E675E0CE014C
:103260000E941A30892B19F40E94D904F2CF80E011
:10327000F1CF611106C065E575E08BEE93E00C942B
:103280001F276BE575E0F9CF109266030895CF9381
:10329000DF93EC018BEE93E00E9441258BEE93E0EF
:1032A0000E944425892B09F45BC08BEE93E00E94B9
:1032B0005425E8A191E09E0F98A3EC0FFD2FF11D7E
:1032C0008083FE01E90FF11D31978081803271F01A
:1032D000903260F48BEE93E00E944425892B31F00C
:1032E0008BEE93E00E942B250A97F9F688818111D5
:1032F00007C018A280E2FE0111928A95E9F730C05A
:10330000E8A1EC0FFD2FF11D319780818032F9F497
:10331000E8A1E150FF0BEC0FFD1F8081803209F422
:103320001082CE010E947F058BEE93E00E9444251F
:10333000892B31F08BEE93E00E9454258A30A1F75F
:1033400064E975E08BEE93E00E944E27D2CF8BEEBE
:1033500093E00E942B250A97D9F288A18032C0F60B
:1033600080E0DF91CF91089568E975E08BEE93E0FE
:103370000E941F2784E690E00E946D046AE08BEEB5
:1033800093E00E94432784E690E00E946D0480E071
:103390000895CF93DF9300D000D000D0CDB7DEB733
:1033A00080ED94E00E94A82EE4EEF4E0108A868579
:1033B00097852485358519823B832A839D838C8359
:1033C0001E820284F385E02D0190F081E02D46E01D
:1033D00050E0BE016F5F7F4F8EEE94E0099580E074
:1033E00026960FB6F894DEBF0FBECDBFDF91CF910A
:1033F0000895FC01703579F4862F8076803429F4A5
:103400009085862F8F7B892B8087862F807729F464
:103410008781682B678380E008958031E1F780E140
:10342000689FB0011124F4CFCF93DF93EC0180EDBE
:1034300094E00E946B2E688580ED94E00E94712ECE
:1034400080ED94E0DF91CF910C94832EFB0192816B
:1034500096FB222720F980E090FD82E0822B20E07D
:1034600091FD24E0822B20E092FD28E0822B93FD49
:1034700004C090E0892B0C94711B90E1FBCFFB0101
:103480002381203559F4DC0117961C92179722816D
:10349000322F3076303421F418961C9280E0089553
:1034A00025FFFCCF218121FFF9CF20FDF7CF0E941E
:1034B000261AF4CF2091B7013091B801FC01318375
:1034C00020839681892F8F7019F4109272030895CA
:1034D00080910F01819592FF80E093FF03C02091BE
:1034E0000F01820F60910F01619590FF60E091FFE5
:1034F00003C090910F01690F0E94131C80ED94E0AE
:103500000C94832E0F932091B7013091B801FC01E8
:1035100035832483868190E024E0959587952A95CC
:10352000E1F70097F1F000910901019582FF00E0B9
:1035300083FF03C020910901020F2091090180FF40
:1035400020E081FF03C080910901281B40E060E07A
:1035500080ED94E00E94632E80ED94E00F910C9436
:10356000832E0F910895CF93DF93EC018091B701E3
:103570009091B8012A813B81AC01421B530B9A0107
:1035800040910A0150910B012417350780F09B836D
:103590008A832091720330910C014FEF50E0431B5E
:1035A0005109241715061CF4230F20937203288158
:1035B0003981821B930B20910D0130910E018217EE
:1035C000930718F0CE010E945A1A8091B70190918A
:1035D000B8012C813D81821B930B20910701309112
:1035E00008018217930718F0CE010E94821A80E02A
:1035F000DF91CF9108950F931F93CF93DF93FB013A
:1036000023812035C9F48B01EC01828180768034DE
:1036100019F4CE010E94141A8F818E831F82F80143
:103620008281807779F48091B7019091B8019B8372
:103630008A83CE010E945A1A80E0DF91CF911F91B8
:103640000F9108958031C1F7CE010E94821AF4CF04
:10365000CF93DF9300D000D000D0CDB7DEB7369542
:103660002795820F931F56954795640F751FE4EEBB
:10367000F4E09587848777876687208929839B83F1
:103680008A837D836C831E820284F385E02D019002
:10369000F081E02D46E050E0BE016F5F7F4F8EEE7F
:1036A00094E0099526960FB6F894DEBF0FBECDBF05
:1036B000DF91CF91089510927503109274031092C8
:1036C0007703109276038FEF9FE790937B038093AD
:1036D0007A03909379038093780381E08093730356
:1036E00008950F931F93CF93C82F80917303811177
:1036F00002C00E945B1BC0FF06C010927303CF91F3
:103700001F910F910895E09111010E2F10E080910B
:103710007A0390917B03B8010E948F2F9B017093D5
:103720007B0360937A038091780390917903B801C9
:103730000E948F2FAB0170937903609378036C2FF5
:103740006470E0917603F091770380917403909117
:1037500075037C2F7670763091F4820F931F9093CF
:10376000750380937403BA016E0F7F1F7093770304
:1037700060937603CF911F910F910C94281B6623C1
:1037800049F1D8011197A49FB001A59F700DB49F76
:10379000700D1124E60FF71FF0937703E093760383
:1037A000C4FF1DC001501109029FB001039F700D9D
:1037B000129F700D1124860F971F909375038093AD
:1037C00074036091760370917703809174039091F4
:1037D0007503D0CFC1FDE4CFE40FF51FDDCFC3FDEE
:1037E000F0CF820F931FE9CF482F50E087FD0AC02A
:1037F000889FC0011124880F892F881F990B9195EC
:103800008F5F089520E031E0241B350B229FC0011B
:10381000239F900D900D1124880F892F881F990BDD
:10382000919580950895EF92FF920F931F93CF93F8
:10383000DF93082F162FC0911001D0E0F12CE12C5E
:103840008823D1F0809172030E94F41B20917103B0
:10385000382F0303C0011124820F911D27FD9A9573
:103860007E01C817D90744F0EE24FF24EC1AFD0AA4
:10387000E816F9060CF47C01112309F449C0809183
:1038800072030E94F41B20917003382F1303C001B0
:103890001124820F911D27FD9A95C817D9073CF076
:1038A000D195C195D109C817D9070CF4EC01109234
:1038B0007303AE01D7FF02C0415F5F4F94E055959F
:1038C00047959A95E1F7B701F7FE02C0615F7F4F18
:1038D00084E0759567958A95E1F700E020E080ED3A
:1038E00094E00E94632E20E130E0C701B9010E94FC
:1038F000A32F80937103CE01B9010E94A32F80935F
:103900007003DF91CF911F910F91FF90EF90089579
:10391000D0E0C0E0CCCFFC018281DB019C91891713
:1039200030F5A081B181A80FB11D2C9130E09381B9
:1039300002C0359527959A95E2F724834481442364
:1039400091F0242F30E0938140FF07C0880F880F4B
:10395000880F890F858381E0089535952795248305
:103960009F5F9383EBCF8F5F82831382D5CF80E0FD
:103970000895262F269526952695820F911DFC01E8
:10398000808190E0677002C0959587956A95E2F70F
:1039900081700895E62FE695E695E695E80FF92FF4
:1039A000F11D677081E090E0A0E0B0E004C0880FF6
:1039B000991FAA1FBB1F6A95D2F72081822B808393
:1039C0000895E62FE695E695E695E80FF92FF11DA7
:1039D000862F877041E050E060E070E004C0440F43
:1039E000551F661F771F8A95D2F7409550956095B1
:1039F00070958081482340830895EF92FF920F9342
:103A00001F93CF93DF93CDB7DEB72C970FB6F89403
:103A1000DEBF0FBECDBF8C010A9698878F831986B3
:103A20001A86FF24FA94FC869A83898386E0E82E1E
:103A3000EB821C82FE82BE016D5F7F4FCE01079636
:103A40000E948B1C811113C0005F1F4F18870F83CA
:103A500019861A86FC861A830983EB821C82FE82F1
:103A6000BE016D5F7F4FCE0107960E948B1C2C9686
:103A70000FB6F894DEBF0FBECDBFDF91CF911F917F
:103A80000F91FF90EF900895272F207C69F4605EDE
:103A9000683098F4FC018681978102C096958795DD
:103AA0006A95E2F781700895743439F426ED260F93
:103AB0002A3218F46252603168F381E008950C9460
:103AC000441DAF92BF92DF92EF92FF920F931F932C
:103AD000CF93DF93CDB7DEB761970FB6F894DEBF13
:103AE0000FBECDBF8C010A967C01662381F158017F
:103AF00090E1A90EB11CB886AF8219861A868FEFA5
:103B00008C87BA82A98296E09B831C828E83BE0139
:103B10006D5F7F4FCE0107960E948B1C8823B9F002
:103B2000DC846D2DC5010E94E11C6D2DC7010E9432
:103B3000E11C609152042D2D31E84FEF5FEF86EBD1
:103B400091E00E9457098A858F5F8A87E0CFF886C7
:103B5000EF8219861A868FEF8C87FA82E98296E0C7
:103B60009B831C828E83005F1F4FBE016D5F7F4F62
:103B7000CE0107960E948B1C882309F1DC846D2DF1
:103B8000C8010E94B91C6D2D8823A9F0C8010E94AC
:103B9000E11C6D2DC7010E94E11C609152042D2D86
:103BA00031E84FEF5FEF86EB91E00E9457098A857D
:103BB0008F5F8A87DACFC7010E94E11CF8CF619638
:103BC0000FB6F894DEBF0FBECDBFDF91CF911F912E
:103BD0000F91FF90EF90DF90BF90AF90089562EA51
:103BE00075E08BEE93E00E941F2784E690E00E9430
:103BF0006D046AE08BEE93E00E94432784E690E038
:103C00000E946D0480E008954F925F926F927F92C0
:103C10008F929F92AF92BF92CF92DF92EF92FF92DC
:103C20000F931F93CF93DF93CDB7DEB761970FB696
:103C3000F894DEBF0FBECDBF8C01FC0160807180A7
:103C4000C090B701D090B80186899789C81AD90A5F
:103C5000828093807801FAE0EF0EF11CF886EF8203
:103C600019861A868FEF8C87FA82E98296E09B8309
:103C70001C828E83512C580180E1A80EB11CBE011C
:103C80006D5F7F4FCE0107960E948B1C482E8823C4
:103C900049F15C84652DC5010E94B91C8823D1F0CF
:103CA000C614D70490F0652DC5010E94E11C652D56
:103CB000C7010E94E11C60915204252D31E84FEFAD
:103CC0005FEF86EB91E00E9457098A858F5F8A87B4
:103CD000542CD5CFC814D904C0F3652DC7010E9458
:103CE000E11CF3CF511007C08091B7019091B8014A
:103CF000F801978B868B80E061960FB6F894DEBF53
:103D00000FBECDBFDF91CF911F910F91FF90EF902C
:103D1000DF90CF90BF90AF909F908F907F906F90EB
:103D20005F904F9008950C94041E872F90E0982F79
:103D30008827860F911D2FEF280F283018F4815205
:103D400090E008958F5D94E40895AF92BF92CF9272
:103D5000DF92EF92FF920F931F93CF93DF93FB01BC
:103D6000B180B7FC5BC0EB018C016C01FAE0CF0EB7
:103D7000D11C6881C6010E94B91CA82E780180E17F
:103D8000E80EF11C6881C7010E94B91CB1FE90C009
:103D9000B0FC8EC0A11051C0811185C08A819B8169
:103DA000292F30E0322F2227482F50E04150504C2D
:103DB000240F351F2031310598F46A817B81C801B9
:103DC0000E94951E9B838A836881C6010E94CA1C3B
:103DD0008091B7019091B801F801978B868B1BC039
:103DE000F8012085222339F0292F207C21F420E2BC
:103DF000280F283048F3F8012185222331F094342C
:103E000021F426ED280F2A32F8F2292F207C41F4E4
:103E1000805E883050F48881F801808F80E038C05F
:103E2000943419F48A528A32B0F3F801868997895A
:103E300020813181821B930BD0CF882361F368816D
:103E4000C6010E94E11C9881F801808D981729F025
:103E50006881C7010E94E11CDECF6A817B81C801B5
:103E60000E945F1D8823A1F3F8018481958197FF4B
:103E700002C0808191812091B7013091B801F80191
:103E800046895789241B350B2817390708F782E024
:103E9000DF91CF911F910F91FF90EF90DF90CF9026
:103EA000BF90AF9008956881C6010E94E11CD0CFF9
:103EB000A11003C0882309F4B1CF6881C7010E9413
:103EC000CA1CE5CF6AEA75E08BEE93E00E941F27DB
:103ED00084E690E00E946D046AE08BEE93E00E941D
:103EE000432784E690E00E946D0480E00895FC0181
:103EF000872F90E0982F8827680F792F711D6131E7
:103F000080EC7807E0F0623188EC780750F461517A
:103F1000704C66A717A611AA80EE870F80AB81E0D0
:103F20000895633180ED780750F46251784C66A7AC
:103F300017A68AE2870F80AB84E481ABF0CF80E0E4
:103F400008958F929F92AF92BF92CF92DF92EF929D
:103F5000FF920F931F93CF93DF9300D000D0CDB784
:103F6000DEB78C01F62E2FE2261708F469C0E62F83
:103F7000F0E0EE0FFF1FED5AFB4FD080E1808FEF96
:103F8000D8120FC0E8120DC0AF2DB0E0A454BE4F40
:103F9000E0910201F09103016F2D8C910995D82ECB
:103FA000E92E6D2D7E2DC8010E94771FB82E81113C
:103FB00035C0EF2DF0E0E454FE4F8080C12CAA24E0
:103FC000AA94912CF8018281C81608F042C0F4E04E
:103FD000CF9EC0011124F80160817181680F791FA3
:103FE000AA8244E050E0CE0101960E9411308981FE
:103FF0009A813B812C81F9122AC0482F082E000C8F
:10400000550B4815590511F08F3F09F5F801D6A653
:10401000E7A6C90190AB21ABBB24B3948B2D0F90C5
:104020000F900F900F90DF91CF911F910F91FF9004
:10403000EF90DF90CF90BF90AF909F908F900895BA
:104040001092B3041092B404E3EBF4E096CFC3945F
:10405000B9CFD6A6E7A68FEF80AB81ABDFCFCF93EA
:10406000DF93FC01EB019A01261B370BA4E6B0E0BD
:104070000E94DF2F26A130E050E040E00E94B72FE1
:104080008091B7019091B801BC016C1B7D0B81E060
:104090006217730708F080E0DF91CF910895292F10
:1040A000207C39F490E2980F81E0983048F080E06D
:1040B00007C09434E1F796ED980F81E09A32B8F793
:1040C0000895CF93DF93EC018881681780F58823EA
:1040D00071F181508883E62FF0E0DF011196AC0F7B
:1040E000BD1FEE0FFF1F7196EC0FFD1F962F981747
:1040F00080F411962C9111972D9318962C91189766
:1041000017962C93179722813381219331939F5FC8
:10411000EECF2FEF30E001C0220F6A95EAF789A1B8
:10412000922F9095982386958223892B89A3DF91DE
:10413000CF910895CF93DF9300D000D01F92CDB7D9
:10414000DEB7FC01348584A1982F917080FD28C0D2
:1041500082E0248139838A836B837C832D83911150
:104160000AC0872F90E0982F8827680F792F711D3C
:1041700064307105F0F460E0CF0103960E94612085
:1041800029813A814B815C816D8186EB91E00F90B2
:104190000F900F900F900F90DF91CF910C940B0A1E
:1041A00081E0D7CF6D32710530F36933710518F7AF
:1041B00003C068327105B0F78489958994A783A7F5
:1041C000DACFCF93DF93FC017381DC011D9681E090
:1041D00090E060E08717F0F452A94D9124A130E0FF
:1041E000082E02C0359527950A94E2F720FD0DC0F0
:1041F000541721F080E0DF91CF910895248935890B
:1042000034AB23AB682F0196E5CF5413FCCF8FEF6F
:1042100082ABF0CF8091B7019091B80123A934A966
:10422000821B930B25A92817190609F068F48FEF54
:1042300082AB6623F9F2EF012396CE010E94612042
:1042400060E0CE010E94612081E0D5CF7F928F9205
:104250009F92AF92BF92CF92DF92EF92FF920F9315
:104260001F93CF93DF93EC019B81911110C0F12C30
:104270008F2DDF91CF911F910F91FF90EF90DF90E5
:10428000CF90BF90AF909F908F907F9008959C8427
:104290008CA180FF13C0983041F460E070E0CE0143
:1042A0000E949A20FF24F394E3CF8AA99812F5CFB5
:1042B000CE010E94E1208111DACFEFCF692DCE012E
:1042C0000E94A11F882309F470C0FDA0FF2009F4FB
:1042D0006CC00EA51FA5C8010E944F20882E80919A
:1042E000B7019091B8012BA53CA5821B930B2AA581
:1042F0002817190609F010F57B80A090B701B0903F
:10430000B8016E0101E010E0E12C202F071508F044
:1043100065C08CA190E0002E02C0959587950A9407
:10432000E2F780FD12C0811040C0EE2009F454C0B5
:104330007FEFC71AD70A0F5F1F4FE7CF8110DCCF7F
:10434000B801CE010E949A20D7CFF6019585FE01D3
:104350003D9681E099122DC0EE2019F08EA18111B9
:1043600010C0882059F068A979A99AAA8C899D89DA
:104370009CAB8BABCE010E949A207ACF6EA57FA515
:10438000F4CFF801EE0FFF1FEC0FFD1F4489558994
:10439000EE2DF0E0EE0FFF1FEC0FFD1F6489758915
:1043A000CE010E942F208111C3CF6EA57FA577CFAC
:1043B0008F5F821708F0BCCF31913913F9CF4C8948
:1043C0005D89B501641B750B39A53617170609F011
:1043D00078F768A979A9CECFE02EAACF88E0781225
:1043E00046CFE3CF0F931F93CF93DF93EC01FB01F5
:1043F00024818DA5922F981B19162CF08B81811189
:104400001CC080E025C02DA780818033D0F781813A
:1044100087FDF7CF8B018DA181111FC06281738150
:10442000CE010E94771F882361F38EA59FA5D80136
:1044300013969C938E931297E4CF022E000C330BAD
:104440008C81281B310987FD339537FDDACF82E057
:10445000DF91CF911F910F9108952B81822F90E0D2
:104460003481FE01E80FF91F3483DB013C9134876E
:10447000880F991FFE01E80FF91F8091B7019091F5
:10448000B801958B848B11964C913CA181E090E012
:10449000A0E0B0E0022E04C0880F991FAA1FBB1F26
:1044A0000A94D2F740FF0CC041FD0AC0832B8CA3B5
:1044B0002F5F2B83CE010E9426218111FBCFC7CF16
:1044C00080958323F4CF0F931F93CF93DF93EC0159
:1044D0002091B7013091B8018AA590E04BA55CA569
:1044E000B901641B750B6817790738F0A9014150B1
:1044F0005109481B590B5CA74BA78B818823D9F026
:104500008C899D89281B390B8FA198A528173907FD
:1045100068F00EA51FA5C8010E944F20B8018111A7
:1045200002C068A979A9CE010E949A20CE010E94FA
:1045300026218111FBCF80E0DF91CF911F910F9158
:104540000895CF93DF93CCE7D3E0198218821A82C3
:104550001B8288E0E0E4F1E0A8E8B3E001900D926E
:104560008A95E1F781E08DA380E58EA38AEF90E044
:1045700098A78FA382E389A78BE48AA780E091E0C4
:104580009CA78BA78FEF8DA78EA78FA788AB89AB32
:104590008AAB88EC8DABDF91CF910895FC018FEF52
:1045A00081831282409148015091490160914A01F2
:1045B00070914B014783508761877287848B80910C
:1045C000C70381112CC081EE8093CF031092D003DA
:1045D00086E28093D10388E08093D2031092D403C3
:1045E0001092D30395EE9093D5031092D60397E2E1
:1045F0009093D7038093D8031092DA031092D903D3
:104600001092DB031092DC031092DD031092DE03A4
:104610001092E0031092DF0381E08093C7038FECD8
:1046200093E09093E2038093E103089561EB75E0DA
:104630008BEE93E00E941F2784E690E00E946D04B9
:104640006AE08BEE93E00E94432784E690E00E94AC
:104650006D0480E0089580E026E0E091E103F091B0
:10466000E203829FE00DF11D1124908191110FC092
:10467000318131110CC03281311109C033813111C6
:1046800006C044815581452B11F48FEF0895961390
:1046900003C09181971711F08F5FDFCF08950F93BB
:1046A0001F93CF93DF93CDB7DEB72A970FB6F89459
:1046B000DEBF0FBECDBF8C01FC01838980FD48C0E9
:1046C00082E0F801278193812E838F838FEF888783
:1046D00089879A87662321F1948997FD21C090816B
:1046E000923079F460915204298391E09A838B830C
:1046F0008C836D8331E04FEF5FEF86EB91E00E949A
:104700005709F8018489E091E103F091E20396E012
:104710008902E00DF11D1124828193819987888798
:10472000F80182818823E1F0815082833396D80199
:104730001B9690E0981770F42181219324812383A4
:1047400012962D913C9113972D933D939F5FF2CF3D
:1047500081E0B7CFF801838990E095958795838BA9
:104760002E813F81488559856A8586EB91E02A969E
:104770000FB6F894DEBF0FBECDBFDF91CF911F9172
:104780000F910C940B0ACF93DF93EC018A8188235D
:1047900029F060E0CE010E944F23F8CFDF91CF9146
:1047A0000895FC018281882311F120912B01309121
:1047B0002C018489A091E103B091E20396E0890283
:1047C000A00DB11D112414968D919C91009709F0B4
:1047D0009C018091B7019091B80143855485841B59
:1047E000950B8217930718F0CF010E94C32380E036
:1047F0000895CF93DF93FC01EB012081822F90E09D
:104800003C81DF01A80FB91F11963C9311973881A5
:1048100015963C93880F991FDF01A80FB91F80914F
:10482000B7019091B8011A969C938E93199799812C
:10483000818941E050E060E070E0022E04C0440F46
:10484000551F661F771F0A94D2F790FF09C091FD8C
:1048500007C0482B418B2F5F2083DF91CF910895B4
:1048600040954823F7CF0F931F93CF93DF93EC012D
:10487000FB0184819981282F291B12164CF09A8103
:1048800091111CC080E0DF91CF911F910F9108958D
:10489000898320812033B0F7818187FDF3CF382FC2
:1048A000327081FF1FC080FD1DC09281983591F448
:1048B0009381913DB9F4188281E0E5CF082E000C78
:1048C000990B2B81821B910927FD939597FDDACFD8
:1048D00082E0D9CF993531F49381913D19F481E08B
:1048E0008883D1CF9881913069F28F019A81992381
:1048F00071F080FF09C0311107C08F81821323C07E
:1049000061E0CE010E944F23CE010E94C323F80133
:10491000818181FFB7CF80FDB5CF62817381CE01E8
:104920000E942B238C8B87FDADCF8881823069F468
:10493000F8012081318142815381648186EB91E0CD
:104940000E94570902C09430F9F2B801CE010296D4
:104950000E94F923BDCF82EB93E00C94CE226CEB46
:1049600075E08BEE93E00E941F2784E690E00E94A2
:104970006D046AE08BEE93E00E94432784E690E0AA
:104980000E946D0480E00895FB012381822F90E056
:10499000982F88272281280F392F311DC9018D5268
:1049A000914D8A9708F03FC081819091EA0381FF81
:1049B0001FC080FD1DC083ED820F9F5F9093EA03AF
:1049C00067E00E94832FE82FF0E0EC51FC4F26E0D7
:1049D00030E0291B310981E090E0AC0102C0440FB6
:1049E000551F2A95E2F78081842B808381E008950A
:1049F0008FEF890F8093EA038111F8CF8091E40350
:104A000080688093E40346E050E064EE73E08BEE50
:104A100093E00E946125E4EEF3E086E0DF011D9261
:104A20008A95E9F7E3CF80E00895CF93DF931F9253
:104A3000CDB7DEB76983DC01ED91FC910280F38193
:104A4000E02D41E050E0BE016F5F7F4F09950F9070
:104A5000DF91CF910895CF93DF93EC018C859D85F5
:104A600097FF05C082E00E9481299D878C878C85F5
:104A70009D85DF91CF91089583E00E94982990E071
:104A8000089583E00C94072CFC018485958597FD9F
:104A900006C082E00E94312990E00196089582E0EC
:104AA0000E94312990E00895FC018485958597FD49
:104AB00005C02FEF3FEF35872487089582E00C94DF
:104AC0008129CF93DF93EC0180913801882331F065
:104AD00083E00E94B2291816190634F081E090E0B4
:104AE0009B838A8380E090E0DF91CF910895EEEF81
:104AF000FFE72591349181E02B3F3C4D09F080E0A8
:104B00000895FC0190819E5F908342E450E065EC43
:104B100075E080E80C94632AFC0181819081913AD0
:104B200061F4813209F083C047E050E061E371E055
:104B300080E00E94632A81E00895913209F077C0F5
:104B4000833269F482819381B0E0A0E080932D01EB
:104B500090932E01A0932F01B0933001ECCF8032BF
:104B600039F467E070E081E391E00E94892AE3CFA5
:104B7000823209F78281809338010E947725E0E034
:104B8000F8E0882311F0EEEFFAE080913101909186
:104B90003201A0913301B0913401803B9440A105D2
:104BA000B105D9F48091380180FD17C0EE3F8AE04D
:104BB000F80771F587E797E791838083809160001C
:104BC00080933B0488E19BE00FB6F894A89580930E
:104BD00060000FBE90936000AECF808191818737D7
:104BE000974709F0A8CFA8958091600088618093CD
:104BF000600080913B0480936000EE3F8AE0F807FC
:104C000089F08091FE0A9091FF0A9183808393CF6F
:104C1000808191818737980769F29093FF0A80938A
:104C2000FE0AC8CF1092FF0A1092FE0A84CF80E0DD
:104C300008952FEF3FEFFC01358724870895EBEEB1
:104C4000F3E01382128288EE93E0A0E0B0E0848368
:104C50009583A683B7838BE791E0918380838FEF61
:104C60009FEF958784870895EF92FF920F931F938C
:104C7000CF93DF937B01FC01C281D38110E000E080
:104C8000209791F0E881F9810280F381E02DB7014E
:104C9000CE01099597FD06C0080F191F0884D98514
:104CA000C02DEECF0FEF1FEFC801DF91CF911F9105
:104CB0000F91FF90EF9008950F931F93CF93DF9381
:104CC0008B01FC01C281D381209771F0E881F981C9
:104CD0000480F581E02DB801CE010995009731F4EB
:104CE0000884D985C02DF0CF90E080E0DF91CF918E
:104CF0001F910F9108950F931F93CF93DF938B0113
:104D0000FC01C281D381209771F0E881F98106808E
:104D1000F781E02DB801CE010995080F111D088417
:104D2000D985C02DF0CFF8011082DF91CF911F916E
:104D30000F9108950F931F93CF93DF938B01FC0185
:104D4000C281D381209771F0E881F9810190F081CF
:104D5000E02DB801CE010995811105C00884D985DF
:104D6000C02DF0CF80E0DF91CF911F910F9108957A
:104D7000CF93DF93FC01DB01218114968C91149772
:104D8000820F9927991F08978CF5C281D3812097AC
:104D900031F573836283908112969C9312971396D8
:104DA0002C93139715968C911597890F808380E02B
:104DB00014969C9114978917E8F41696CD91DC917E
:104DC0001797C80FD11D9881C181D0E0C75CDE4F15
:104DD000988391819F5F91838F5FEACFEC018885F3
:104DE00099850097D9F7B987A887D5CF80E0DF915B
:104DF000CF91089581E0FBCF80913C0481110DC0DB
:104E000082E08093440484E0809345041092470438
:104E10001092460481E080933C0484E494E0089579
:104E2000FB0101900020E9F73197AF01461B570BBA
:104E3000DC01ED91FC910280F381E02D0994EF9269
:104E4000FF920F931F93CF93DF938C017B01D0E0F0
:104E5000C0E0F701EC0FFD1F6491662361F0D801FB
:104E6000ED91FC910190F081E02DC8010995892B0D
:104E700011F02196EECFCE01DF91CF911F910F91CE
:104E8000FF90EF900895DC01ED91FC910190F0818D
:104E9000E02D099469E871E00C9410270F931F939B
:104EA000CF93DF93EC010E941F278C01CE010E945B
:104EB0004A27800F911FDF91CF911F910F91089585
:104EC0008F929F92AF92BF92EF92FF920F931F9398
:104ED000CF93DF93CDB7DEB7A1970FB6F894DEBFBF
:104EE0000FBECDBF7C01FA01CB0119A2223008F41C
:104EF0002AE08E010F5D1F4F822E912CB12CA12C28
:104F0000BF01A50194010E94B72FF901CA016A30BF
:104F10000CF5605DD8016E938D01232B242B252B7E
:104F200079F790E080E0109721F0BD01C7010E9461
:104F30001027A1960FB6F894DEBF0FBECDBFDF914C
:104F4000CF911F910F91FF90EF90BF90AF909F90E6
:104F50008F900895695CDECF2115310541F4DC01A5
:104F6000ED91FC910190F081E02D642F09940C9457
:104F700060279A01462F50E070E060E00C94AC2767
:104F80009A01AB0170E060E00C94AC270F931F9383
:104F9000CF93DF93EC010E940304688779878A87A7
:104FA0009B87E881F9810484F585E02DCE01099580
:104FB00097FF15C00E940304088519852A853B8543
:104FC000601B710B820B930B0C811D812E813F8125
:104FD000601771078207930720F38FEF9FEFDF9130
:104FE000CF911F910F910895FF920F931F93CF932D
:104FF000DF93EC018B01F42ECE010E94C62797FDB2
:105000001DC08D329105D1F09C01205331092A3009
:105010003105A0F0FF2019F08E32910579F00130B2
:10502000110551F00230110589F48D30910571F0B0
:105030005CF40997029750F08FEF9FEFDF91CF91CB
:105040001F910F91FF9008958097B1F7E881F98142
:105050000284F385E02DCE010995CECFBF92CF9289
:10506000DF92EF92FF920F931F93CF93DF938C0108
:10507000C42F40E00E94F427FC01C12CD12C760102
:1050800097FD3EC0B12C0C2E000CDD0BCE17DF07B8
:10509000D9F0ED32F10509F43FC0CF01C0970A976E
:1050A00098F4AAE0B0E0A70196010E94EE2F6F01EC
:1050B000FF0FEE08FF08C60ED71EE81EF91E80E39C
:1050C000C81AD108E108F108D801ED91FC910284D9
:1050D000F385E02DC8010995C8010E94C627FC018F
:1050E000C0970A9798F2CE17DF0781F2BB2041F0F4
:1050F000F094E094D094C094C11CD11CE11CF11C2C
:10510000C701B601DF91CF911F910F91FF90EF90F2
:10511000DF90CF90BF900895BB24B394D5CF40913A
:105120004B0450914C042091490430914A04421799
:105130005307B4F49091E8009570E1F39091E80082
:1051400092FD19C08093F10080914B0490914C0422
:1051500001968F739927892B19F48EEF8093E800BD
:1051600080914B0490914C04019690934C04809351
:105170004B0481E0089580E00895EF92FF920F9331
:105180001F93CF93DF93F82E192FE62E042F81E083
:10519000860F880F0E948F2883E00E948F28CF2DD2
:1051A000D12FEC0EFD2EF11CCE15DF05B9F007FF57
:1051B00013C0FE0184910E948F28182F80E00E9466
:1051C0008F28812321968111EFCFDF91CF911F91FD
:1051D0000F91FF90EF9008958881EDCF81E0F5CF9A
:1051E0008091D70081608093D70080EA8093D800B7
:1051F00089B5806189BD89B5826089BD09B400FE29
:10520000FDCF61E070E080E090E00E943404809186
:10521000D8008F7C80618093D8008091E000807FEF
:105220008093E0000895CF93DF931F92CDB7DEB750
:105230001982CE0101960E9481250E94FC26BE01A2
:105240006F5F7F4F0E94342689810F90DF91CF914D
:1052500008952FB7FC012083F89467706093E900EC
:105260000895CF93DF931F92CDB7DEB7682FCE019D
:1052700001960E9429298091F20099819FBF0F9089
:10528000DF91CF910895EF92FF920F931F93CF93E9
:10529000DF931F92CDB7DEB790914F04992371F140
:1052A00057FD2CC08A017B01682FCE0101960E9418
:1052B00029298091F20090E0081719070CF4C80121
:1052C000282FF70144E6215030F0409350043091EC
:1052D000F1003193F8CF009739F02091F2002111BD
:1052E00003C02BE62093E80029812FBF0F90DF91A8
:1052F000CF911F910F91FF90EF9008958FEF9FEF47
:10530000F5CFCF93DF931F92CDB7DEB741E050E0EA
:10531000BE016F5F7F4F0E944329019731F489815D
:1053200090E00F90DF91CF9108958FEF9FEFF9CF2D
:10533000CF93DF931F92CDB7DEB7682FCE010196D2
:105340000E9429299091E800892F807295FF04C05E
:105350009091F20080E4891B99819FBF0F90DF91AB
:10536000CF9108955F926F927F928F929F92AF92AA
:10537000BF92CF92DF92EF92FF920F931F93CF9342
:10538000DF931F92CDB7DEB7982E6B01B42E052F99
:1053900080914F04811113C08FEF9FEF0F90DF9129
:1053A000CF911F910F91FF90EF90DF90CF90BF9022
:1053B000AF909F908F907F906F905F9008958091B5
:1053C0004D0480FF05C08091E00082608093E00082
:1053D000EB2CF02EA12C8AEF882E892D8072682E5E
:1053E000892D8074582E9AE3792EE114F10419F472
:1053F000AA2009F457C0892D0E949829182F8111DD
:105400000AC08A94882041F261E070E080E090E078
:105410000E943404EACF8E151F0411F00CF01E2DEB
:10542000692DCE0101960E9429298091E80085FD11
:1054300003C089818FBFD9CF812F90E0E81AF90A84
:10544000662029F01150A0F01092F100FBCFF60178
:1054500097FC0AC0115050F021912093F100FACF2F
:1054600024912093F10031961150D0F7C80ED91E27
:10547000AA2021F07092E800A12CDBCF8091E800F7
:1054800085FD08C07092E800AA24A394E114F104F9
:1054900081F2F2CFE114F10461F6552051F27092DD
:1054A000E800C7CF84E6809351048B2D902F76CFF0
:1054B0001092E90010924C0410924B0490934A040D
:1054C000809349040895DF92EF92FF920F931F9308
:1054D000CF93DF93D82E8A01EB017B01E40EF51EFA
:1054E000CE15DF0559F0D7FE12C0FE0184910E944F
:1054F0008F2821968111F4CF0FEF1FEFC801DF91A4
:10550000CF911F910F91FF90EF90DF9008958881C8
:10551000EECFCF93DF93EC019B01B4E6ABEF211507
:105520003105F1F0A9012134310514F040E450E0D7
:105530008091E80082FFFCCF942FFB01E21BF30B6C
:10554000EC0FFD1F915028F08091F100808331967F
:10555000F9CFB0935004A093E800241B350BDFCFA4
:10556000CB01DF91CF9108951F920F920FB60F924A
:105570001124CF92DF92FF920F931F932F933F93AB
:105580004F935F936F937F938F939F93AF93BF934B
:10559000EF93FF93CF93DF93CDB7DEB76C97DEBF6A
:1055A000CDBF1092E9008091E80083FF2FC089E011
:1055B000FE017596FE2E0F2F815029F09091F1007B
:1055C00090833196F9CF84E68093500482EF8093E4
:1055D000E8008D8987FF38C09091E80090FFFCCFEC
:1055E000982F907609F000C19E894F89588D2F8998
:1055F000188D911130C0803859F580914E048093F8
:10560000F1001092F1008EEF8093E8006C960FB6D7
:10561000F894DEBF0FBECDBFDF91CF91FF91EF9128
:10562000BF91AF919F918F917F916F915F914F91BA
:105630003F912F911F910F91FF90DF90CF900F908E
:105640000FBE0F901F9018959EEF9093E800C8CF63
:105650001092F100D6CF913059F48111D4CF41305E
:10566000510589F680914E048D7F80934E04CBCFF7
:10567000933049F48111C7CF4130510521F6809113
:105680004E048260F2CF953041F48091E80080FFB3
:10569000FCCF20682093E300B6CF963009F076C0A7
:1056A000CB8CDC8C123039F590E080E00E94582AD7
:1056B0000E9413291F8299E099831A8391E09E83A7
:1056C00090EA98879AEF998720914B0430914C0487
:1056D000275F3F4F3C832B838D83C6010E94582A4E
:1056E00049E050E0BE016F5F7F4F80E00E94632A77
:1056F0000E94132988CFC6010E94582A0E94FC26C6
:105700006F2D702F0E945C26009731F00CF07BCF3C
:1057100081E28093EB007ACF113061F11330C1F751
:105720008F89882381F1823049F440E86CE083E27C
:1057300096E00E94BD28882359F365CF813029F473
:1057400040E869E089E196E0F4CF833009F70E94F0
:10575000FC268E010F5F1F4FB8010E947B26F801C7
:1057600001900020E9F73197BF01601B710B40E009
:10577000C801DFCF67E076E0FB01449150E080E8AC
:105780000E94632A40CF60E376E0F6CF973009F4B9
:10579000BFCF983021F481E08093F10034CF99306D
:1057A00009F031CF837009F0B3CFEAE3F1E081E093
:1057B00031E096E32191222371F08093E900309348
:1057C000EB00DF0111972C912093EC009093ED00FA
:1057D0008F5F873079F78EE78093EA001092EA00B6
:1057E0008F8980934F040FCF8B8D9C8D0E94582AF8
:1057F000898D811105C08F2D902F0E948C259BCF04
:105800000E94FC266F2D702F0E949A2694CF8093C1
:10581000E9008091F200882319F08AE38093E80080
:1058200008951F920F920FB60F9211242F933F935A
:105830004F935F936F937F938F939F93AF93BF9398
:10584000CF93EF93FF93C091E1008091E100837FBC
:105850008093E100C3FF0FC01092E90081E08093C4
:10586000EB001092EC0082E38093ED0010924F0465
:1058700088E08093F000C2FF15C083E00E94072CEF
:1058800080915104882329F08091510481508093A4
:10589000510480915004882329F080915004815054
:1058A00080935004C4FF23C08091E2008E7E81600B
:1058B0008093E2008091E1008F7E8093E1008091EF
:1058C0004D048E7E806180934D04FF91EF91CF91C6
:1058D000BF91AF919F918F917F916F915F914F9108
:1058E0003F912F910F900FBE0F901F901895C0FF02
:1058F000ECCF8091E2008E7E80618093E200809107
:10590000E1008E7E8093E10080914D048E7E816067
:10591000DACF10924F0410924E0410924D040E9460
:10592000F028E1EEF0E080818E7E80838DE0809330
:10593000E200559A209A08958091E0008D7F80932F
:10594000E0008091E00081FD11C080914D0480FF56
:105950000DC080914E0481FF09C00E94F028809103
:10596000E00082608093E00081E0089580E0089587
:1059700008951092B3041092B404089587E090EB58
:10598000DC018093F8049093F904A093FA04B09397
:10599000FB0488E19CE00FB6F894A8958093600022
:1059A0000FBE90936000FFCFCF93DF93CDB7DEB7EC
:1059B00069970FB6F894DEBF0FBECDBFFC01DB01C7
:1059C0008C918F5F8C939E012D5F3F4F8DE0D901AD
:1059D0001D928A95E9F729E0298384E08A8391E082
:1059E0009D8383E08E832A8721E22B879C879D8776
:1059F0009F8722E2288B27E02B8B25E02C8B8E8B38
:105A000020E430E0388F2F8B998F82818B839585AE
:105A10008685998B8A8B838180688D8B49E150E0E4
:105A2000BE016F5F7F4F80E00E94632A69960FB6C8
:105A3000F894DEBF0FBECDBFDF91CF910895EF92F6
:105A4000FF920F931F93CF93DF93FB0120812138A7
:105A5000A1F52381223289F5DC0112964C91248133
:105A600035814217130649F5EC0181E00E94822F2F
:105A70000B851C85F12CE12C0115110589F0F8012D
:105A8000448155816281738180E80E94632A8F3F3F
:105A9000980761F0E80EF91ED8010D911C91ECCF2A
:105AA00081E08F8780E00E94822FC701DF91CF9134
:105AB0001F910F91FF90EF90089590E080E0F6CF56
:105AC000CF93DF93EC01DB012A8114968D919C9199
:105AD00015972817190659F411968C9111979C91D6
:105AE000913A39F4982F9D7F81E0913051F080E018
:105AF00008C09132E1F78B3039F412968C918F8780
:105B000081E0DF91CF9108958A3021F413968C9132
:105B1000888BF6CF893059F716968D919C918230FB
:105B2000910539F462E070E0CE0141960E94892A25
:105B3000DECF0197E1F661E070E0CE0142960E946F
:105B4000892A198AD4CFFC01A385B485109771F4F2
:105B50007487638785859685DB0114962D913C912A
:105B6000820F931F968785870895DC018D919C9104
:105B700011970097D1F76D937C93ECCFAF92BF92C2
:105B8000CF92DF92EF92FF920F931F93CF93DF9309
:105B90001F92CDB7DEB77C0169836A01590141E0EC
:105BA00050E0BE016F5F7F4FFC0183810E94B229EC
:105BB0008C0197FD0BC0F7018381A501B6018064BC
:105BC0000E94B229080F191F97FD8C01C8010F9080
:105BD000DF91CF911F910F91FF90EF90DF90CF90C9
:105BE000BF90AF900895CF92DF92EF92FF921F93F4
:105BF000CF93DF93162F7A0169010E94BE2DEC012D
:105C0000E0916702F0916802309729F09C01A601AB
:105C1000B701812F0995CE01DF91CF911F91FF90A0
:105C2000EF90DF90CF900895CF93DF93EC0181E068
:105C30008C838D839E01265F3F4F3F832E83198681
:105C4000188620E931E0398328831C861B861E864E
:105C50001D868F87888B198A1A8A81EC8A870E9411
:105C6000FC26BE01DF91CF910C94B8268091B5043B
:105C7000811107C08DEB94E00E94142E81E0809387
:105C8000B5048DEB94E00895FC0115828091D60453
:105C9000811113C01092DF041092DE0484E396E0B9
:105CA0009093E1048093E0048AE390E09093E3040E
:105CB0008093E20481E08093D6040E94362E6EED3C
:105CC00074E00C94A32D0F93FC0161834283238322
:105CD00004830F91089525E0FC0111922A95E9F7BC
:105CE0000895FC019081692B60830895CF93DF9321
:105CF000EC010E94362E25E030E0AE0161E0DF913C
:105D0000CF910C94F32DCF93DF93EC0198818D818B
:105D100098130CC08981811109C08A81811106C044
:105D20008B81811103C08C81882329F0CE010E94D0
:105D3000762E88818D83DF91CF910895CF93DF9365
:105D4000EC010E946B2ECE01DF91CF910C94832E3B
:105D50000C949E2E80ED94E00C94442ECF93DF9310
:105D6000CDB7DEB769970FB6F894DEBF0FBECDBFD3
:105D7000FC01DB019C919F5F9C939E012D5F3F4F37
:105D800081E1D9011D928A95E9F729E0298384E010
:105D90008A8391E09D8383E08E832A8721E22B878B
:105DA0009C879D879F8722E2288B25E3298B27E00C
:105DB0002B8B25E02C8B8E8B20E430E0388F2F8BC3
:105DC000998F82818B83838180688D8B49E150E03C
:105DD000BE016F5F7F4F80E00E94632A69960FB615
:105DE000F894DEBF0FBECDBFDF91CF9108950F9322
:105DF0001F93CF93DF93EB018A01FC0183818064C1
:105E00000E94B229E0916702F0916802309749F050
:105E10009C01A801BE0187E0DF91CF911F910F91F6
:105E20000994DF91CF911F910F9108950A970C94D7
:105E3000F72EDC01FB0112962C911297848195813B
:105E40002817190641F491818081813A31F49D7FB0
:105E500081E0913009F080E008958132E1F79B30D4
:105E600029F4828152968C9381E008959A3099F7B3
:105E7000828153968C93F8CFFB0120812138B1F4B5
:105E80002381223299F4DC0112964C9112972481DD
:105E900035814217130651F421E052962C9345E3C5
:105EA00050E06EE676E080E80C94632A90E080E0B3
:105EB0000895CF93DF93EC0181E08C838D839E0165
:105EC0002F5E3F4F3F832E83198618861D861C86C2
:105ED0001F861E86188A2CE931E0398328832AEA36
:105EE00031E03B872A878A8B8B8B81EC898B0E94E0
:105EF000FC26BE01DF91CF910C94B82684EE94E08D
:105F00000C94592F0895991B79E004C0991F961796
:105F100008F0961B881F7A95C9F780950895AA1BEB
:105F2000BB1B51E107C0AA1FBB1FA617B70710F084
:105F3000A61BB70B881F991F5A95A9F780959095B6
:105F4000BC01CD01089597FB072E16F4009407D0ED
:105F500077FD09D00E948F2F07FC05D03EF4909565
:105F600081959F4F0895709561957F4F0895A1E2A7
:105F70001A2EAA1BBB1BFD010DC0AA1FBB1FEE1FC3
:105F8000FF1FA217B307E407F50720F0A21BB30B0E
:105F9000E40BF50B661F771F881F991F1A9469F78A
:105FA00060957095809590959B01AC01BD01CF01E6
:105FB0000895EE0FFF1F0590F491E02D0994A29F24
:105FC000B001B39FC001A39F700D811D1124911DCD
:105FD000B29F700D811D1124911D08950E94DF2F25
:105FE000A59F900DB49F900DA49F800D911D11242D
:105FF00008950024A7FD00942A0F301D401D501D58
:10600000601D701D801D901D08950024A7FD009443
:106010002A1730054005500560057005800590057C
:106020000895FB01DC0102C005900D9241505040E3
:10603000D8F70895FB01DC018D91059080190110BE
:10604000D9F3990B0895FB01DC014150504030F029
:106050008D910590801919F40020B9F7881B990BD0
:106060000895FB01DC0104C08D910190801921F499
:1060700041505040C8F7881B990B0895FB01DC0183
:1060800002C001900D9241505040D8F70895681712
:10609000790768F4FB01DC01E40FF51FA40FB51FBD
:1060A00002C002900E9241505040D8F708950C94CF
:1060B0003E30F999FECF92BD81BDF89A992780B5FF
:1060C0000895262FF999FECF1FBA92BD81BD20BD3C
:1060D0000FB6F894FA9AF99A0FBE01960895F894BB
:0260E000FFCFF0
:1060E20006FF9D0B01290032000140000101000161
:1060F2007F02C409FA00FFFFFFFF0000000000005A
:1061020000000000000000000000FFC800FFFFFFC9
:10611200FF00E100000000000000C18081000000DB
:10612200FFFFFFFFFFFFFFFFFFFFFFFF73706C69C1
:10613200746F67726170687900B601F0F1F4F5F678
:10614200F76766363534979091929300000000818C
:106152000D190D640D120D00000000152561253C7E
:10616200254125442554252B250D0A000000000059
:10617200602DD42C1F2DCF0400000000192FAE2E4D
:0C6182003C2F120DF72EF6FF0000162F28
:00000001FF
